:100000000C9434000C9451000C9451000C94510049
:100010000C9451000C9451000C9451000C94380134
:100020000C9451000C9451000C9451000C94070155
:100030000C9451000C9451000C94D6000C94510077
:100040000C9451000C9451000C9451000C945100EC
:100050000C9451000C9451000C9451000C945100DC
:100060000C9451000C94510011241FBECFEFD8E026
:10007000DEBFCDBF11E0A0E0B1E0E8E3F8E002C0F0
:1000800005900D92A831B107D9F711E0A8E1B1E0D0
:1000900001C01D92AD31B107E1F70E94AE010C9491
:1000A0001A040C940000CF92DF92EF92FF92CF934C
:1000B000DF93EC01C880D980EA80FB8020E030E04B
:1000C00040EC50E4C701B6010E9446020E94EB02D8
:1000D00020E030E040EC50E40E94B7039B01AC010B
:1000E000C701B6010E94DD016B017C0120E030E018
:1000F00040E450E40E94420287FF03C08FEF90E08B
:1001000002C080E090E09D838C8320E030E040E4FA
:1001100050E4C701B6010E94B30318161CF48FEF18
:1001200090E002C080E090E09F838E838E899F895B
:100130008230910561F08330910599F00197C9F4FF
:1001400016BC80916E00826080936E0016C0109283
:1001500085001092840080916F00826080936F0010
:100160000CC01092B2008091700082608093700089
:1001700004C081E090E00E941A0478949FB7F8943C
:1001800080911A019FBF8823C9F310921A01EE854E
:10019000FF858C818083EA89FB898E818083DF9152
:1001A000CF91FF90EF90DF90CF9008951F920F9224
:1001B0000FB60F9211242F933F938F939F938091AB
:1001C00018019091190101969093190180931801DB
:1001D00080911A01813091F020911801309119011C
:1001E00080911B0190911C012817390738F081E09C
:1001F00080931A0110921901109218019F918F910A
:100200003F912F910F900FBE0F901F9018951F9246
:100210000F920FB60F9211242F933F938F939F93BA
:100220008091180190911901019690931901809382
:10023000180180911A01813091F0209118013091BC
:10024000190180911B0190911C012817390738F082
:1002500081E080931A0110921901109218019F9168
:100260008F913F912F910F900FBE0F901F90189577
:100270001F920F920FB60F9211242F933F938F93DB
:100280009F93809118019091190101969093190103
:100290008093180180911A01813091F0209118010A
:1002A0003091190180911B0190911C012817390789
:1002B00038F081E080931A01109219011092180110
:1002C0009F918F913F912F910F900FBE0F901F9094
:1002D0001895CF93DF93FC01C1E8D0E088818D6051
:1002E000888382E090E0918B808B229A40E850E0F6
:1002F000DA012C9121622C932AE830E0D901119681
:100300001C921E921C92338B228B28812D60288395
:1003100095878487219ADA012C9121682C93A8E88B
:10032000B0E011961C921E921C92B787A68725B545
:10033000236025BD21E030E0358B248B90931C0198
:1003400080931B0184B5826084BD89EF87BD378BA4
:10035000268B80E090E0DF91CF910895CF92DF92DD
:10036000EF92FF9280E091E00E946901C12CD12CB4
:10037000760160E070E0CB016093000170930101B1
:10038000809302019093030180E091E00E9453006A
:100390008FEFC81AD80AE80AF80AC701B6010E9406
:1003A000AE022FE632E143E05BE30E94B70320E0B8
:1003B00030E0A9010E94DE01DFCF5058BB27AA27F9
:1003C0000ED080C171D130F076D120F031F49F3F52
:1003D00011F41EF466C10EF4E095E7FB33C1E92F7A
:1003E00082D180F3BA17620773078407950718F064
:1003F00071F49EF5B1C10EF4E0950B2EBA2FA02D2D
:100400000B01B90190010C01CA01A0011124FF27C1
:10041000591B99F0593F50F4503E68F11A16F040BC
:10042000A22F232F342F4427585FF3CF46953795BB
:100430002795A795F0405395C9F77EF41F16BA0B80
:10044000620B730B840BBAF09150A1F0FF0FBB1F2E
:10045000661F771F881FC2F70EC0BA0F621F731F77
:10046000841F48F4879577956795B795F7959E3FD4
:1004700008F0B3CF9395880F08F09927EE0F979562
:1004800087950895BBD008F481E008950CD01AC177
:1004900012D140F009D130F021F45F3F19F0D2C001
:1004A00051115BC1FEC01FD198F39923C9F35523A5
:1004B000B1F3951B550BBB27AA2762177307840757
:1004C00038F09F5F5F4F220F331F441FAA1FA9F30D
:1004D00033D00E2E3AF0E0E830D091505040E695FF
:1004E000001CCAF729D0FE2F27D0660F771F881F60
:1004F000BB1F261737074807AB07B0E809F0BB0B4F
:10050000802DBF01FF2793585F4F2AF09E3F510572
:1005100068F098C022C15F3FECF3983EDCF386950B
:1005200077956795B795F7959F5FC9F7880F911DE8
:100530009695879597F90895E1E0660F771F881FD4
:10054000BB1F621773078407BA0720F0621B730B87
:10055000840BBA0BEE1F88F7E0950895E89409C064
:1005600097FB3EF490958095709561957F4F8F4FE6
:100570009F4F9923A9F0F92F96E9BB279395F695FC
:10058000879577956795B795F111F8CFFAF4BB0F7A
:1005900011F460FF1BC06F5F7F4F8F4F9F4F16C0DE
:1005A000882311F096E911C0772321F09EE8872F68
:1005B000762F05C0662371F096E8862F70E060E024
:1005C0002AF09A95660F771F881FDAF7880F96959D
:1005D000879597F90895A9D080F09F3740F491113D
:1005E0000EF0BBC060E070E080E89FEB089526F459
:1005F0001B16611D711D811D2BC045C0990F000880
:10060000550FAA0BE0E8FEEF16161706E807F907E4
:10061000C0F012161306E407F50798F0621B730B7F
:10062000840B950B39F40A2661F0232B242B252B00
:1006300021F408950A2609F4A140A6958FEF811DA3
:10064000811D089597F99F6780E870E060E0089544
:10065000882371F4772321F09850872B762F07C0D9
:10066000662311F499270DC09051862B70E060E04D
:100670002AF09A95660F771F881FDAF7880F9695EC
:10068000879597F908959F3F31F0915020F4879511
:1006900077956795B795880F911D9695879597F9EA
:1006A00008959FEF80EC089500240A94161617060B
:1006B00018060906089500240A9412161306140653
:1006C00005060895092E0394000C11F4882352F0B6
:1006D000BB0F40F4BF2B11F460FF04C06F5F7F4F6E
:1006E0008F4F9F4F089557FD9058440F551F59F055
:1006F0005F3F71F04795880F97FB991F61F09F3F0F
:1007000079F087950895121613061406551FF2CF37
:100710004695F1DF08C0161617061806991FF1CF87
:1007200086957105610508940895E5DFA0F0BEE7A0
:10073000B91788F4BB279F3860F41616B11D672FD0
:10074000782F8827985FF7CF869577956795B11DA5
:1007500093959639C8F30895E894BB2766277727C1
:10076000CB0197F908954ADF08F48FEF08950BD075
:10077000A9CF9ADF28F09FDF18F0952309F062CF08
:1007800090CF1124EACFAFDFA0F3959FD1F3950F5F
:1007900050E0551F629FF001729FBB27F00DB11D05
:1007A000639FAA27F00DB11DAA1F649F6627B00D95
:1007B000A11D661F829F2227B00DA11D621F739F7E
:1007C000B00DA11D621F839FA00D611D221F749F8C
:1007D0003327A00D611D231F849F600D211D822FD3
:1007E000762F6A2F11249F5750408AF0E1F088231A
:1007F0004AF0EE0FFF1FBB1F661F771F881F915027
:100800005040A9F79E3F510570F01CCFA6CF5F3F27
:10081000ECF3983EDCF3869577956795B795F79559
:10082000E7959F5FC1F7FE2B880F911D96958795E1
:0808300097F90895F894FFCF39
:1008380000000000000000006F12033B00000000F1
:080848000000000000000000A8
:00000001FF
